:100000000C9432000C944F000C944F000C944F0051
:100010000C944F000C944F000C944F000C944F0024
:100020000C944F000C944F000C944F000C944F0014
:100030000C944F000C944F000C944F000C944F0004
:100040000C944F000C944F000C944F000C944F00F4
:100050000C944F000C944F000C944F000C944F00E4
:100060000C944F0011241FBECFEFD8E0DEBFCDBFF0
:1000700011E0A0E0B1E0E2EEF0E002C005900D92E8
:10008000A030B107D9F711E0A0E0B1E001C01D92A6
:10009000A030B107E1F70E9451000C946F000C945E
:1000A00000002F9A279A80E885B928EE33E044E6CD
:1000B00050E060E805C0CA010197F1F721503040D7
:1000C00021153105C1F715B888EE93E0FA01319793
:1000D000F1F70197D9F765B928EE33E0ECCFF89442
:0200E000FFCF50
:00000001FF
